:020000040800F2
:10500000001C0020D55000081D830008017A00080C
:105010000000000000000000000000000000000090
:105020000000000000000000000000009F8D00084C
:10503000000000000000000065830008DD97000804
:10504000E7500008E7500008E7500008E750000864
:10505000E750000891580008F9580008E750000888
:1050600000000000E75000081D580008E750000845
:10507000E7500008E17D000800000000E75000084C
:1050800000000000E75000080000000000000000E1
:10509000E750000800000000E7500008E750000853
:1050A000E7500008E7500008E75000082DA100086D
:1050B000E7500008F17D000800000000000000003B
:1050C0000348854600F04CFB00480047A1AD0008AE
:1050D000001C00200448804704480047FEE7FEE724
:1050E000FEE7FEE7FEE7FEE781980008C1500008F2
:1050F00030B50B46014600202022012409E00D4670
:10510000D5409D4205D31D469540491B25469540F7
:1051100040191546521E002DF1DC30BDF0B51FB40C
:105120000646002082B005464024019100901BE015
:10513000019922460F46304600F020F8049A059B5C
:10514000801A994110D310461946224600F048FAB9
:10515000361A8F410197224601200021009F00F05E
:105160003FFA38184D4100902046641E0028DFDCCD
:10517000019B00982946324607B0F0BD10B5202AA1
:1051800004DB0846203AD040002110BD0B46D34036
:10519000D0402024A21A91400843194610BD03466E
:1051A0000B439B0703D009E008C9121F08C0042A5B
:1051B000FAD203E00B780370401C491C521EF9D24E
:1051C0007047D2B201E00270401C491EFBD270470A
:1051D0000022F6E710B513460A4604461946FFF7C3
:1051E000F0FF204610BD0000F0B5074608465840C5
:1051F00087B0C00F049048000E4659004008490887
:10520000BC1A884105D2384631461E4617460B4621
:1052100002465800400810434CD0300D0390400522
:105220005900400D490D0590401A0290402872DA4D
:1052300018030121000B090508430190049800920E
:10524000002805D001995242002088410092019027
:10525000029840210A1A0199009800F0C1F9054608
:105260000C466B4607CB00F0CBF9C0197141039A8D
:105270000E0D0023D71756401A467A40164344D0E5
:10528000049A002A2DD0029A012A039A15DC1205ED
:10529000C01A914101263605001C7141D20F059EAE
:1052A000D2070093019202962A46234600F0C8F9DD
:1052B00007B0F0BD38463146FAE71605224A0F46D8
:1052C000B218C01AB74101210905001C4F4100184E
:1052D0007F41114618187941E20F10436D1964415E
:1052E00013E0E2076D0815436408C2071443039AEC
:1052F00001261205C01A91413605001C7141CE07E6
:10530000400830434908C01851412A46234600F05E
:105310008AF9CDE7FFE7049801224000C117121A6D
:1053200000238B4104983146C417381AA141EEE797
:1053300030B40124E407634030BC55E730B40124A5
:10534000E407614030BC4FE70000E0FFF0B51FB458
:1053500088B00B990998002448400999C00F49006A
:1053600049080991C0070B990090490049080B9121
:1053700009990898A64608431CD00B990A98084337
:1053800018D0099801244000420D4800410D0998A9
:1053900024050003000B204309900B980003000B29
:1053A00020430B9050181C494018002201901446CD
:1053B000104605E0002001460DB0F0BD032801DADB
:1053C000034600E003239C46C11A0AAE0AE05F00D0
:1053D00008ADED5B4F00F75B7D430027AA187C41C9
:1053E000491C5B1E6145F2DD410004AB5A522104A9
:1053F000120C0A43240C401C0828DFDB01980290A1
:105400000099704601910090059B049A07990698AF
:1054100000F016F9D0E700000DFCFFFFF0B50C46D8
:105420005C4085B0E40FE40703944C000026640858
:1054300059009446490802460296224321D062460A
:105440000A431ED06200570D4A000E032303550D78
:10545000012402462C492405781B1B0B360B4018EF
:1054600023432643614600901C46501AB44103D39F
:105470000098401C009002E0921800985B410028C0
:1054800003DA0020014605B0F0BD00200121090526
:105490000746864611E064461D46141BB54106D3F7
:1054A0006546521BB341744607430C43A646CD07DD
:1054B00040084908284392185B4105460D43EAD14C
:1054C0001046184313D060461946504071400843B7
:1054D00006D06046101AB34106D20122002306E02E
:1054E00000220123DB0702E00122D243531000987F
:1054F00074460105381C6141029C039D00196941F5
:1055000000F091F8BFE70000FD03000070B54B000C
:105510005B0803430BD04B005C0D0026334665420D
:10552000B341D417AD1AA34102DB0020014670BD80
:1055300012053018514170BD0EB5C217C10F504051
:10554000CA0740180021054B0293019200910A46B8
:105550000B4600F075F803B000BD000033040000F6
:105560000EB505490291002100910A460B460191B2
:1055700000F066F803B000BD330400004A000903E0
:105580000123090B1B051943094B10B5520D9A4213
:1055900001DA002010BD064B34339A4203DC9A1A1C
:1055A000FFF7ECFD10BD03495118884010BD000005
:1055B000FF030000CDFBFFFF10B5002904DB012431
:1055C000E40740428C412146002B04DB1C460123AA
:1055D000DB075242A341994200D1904210BD000026
:1055E00010B5202A04DB0146203A9140002010BD6E
:1055F000914020239C1A0346E3401943904010BD7C
:1056000010B5202A06DBCB170846203A1041C117F7
:105610000B4306E00B461341D0402024A21A9140D0
:105620000843194610BD10B5002B08DA0024401CB1
:10563000614192185B411A4301D14008400010BDFE
:10564000F0B51FB482B005460C0003D0084604F044
:1056500095FE02E004F092FE2030024600902146C2
:105660002846FFF7BDFF049B059A04460F461843E2
:105670001143084314D0184610431BD00098402112
:105680000A1A18460599FFF779FD05460E46009A55
:1056900005990498FFF7A4FF084305D0012004E012
:1056A0002046394607B0F0BD0020C11705430E4320
:1056B0002C43374300990E986305401A7905E40A94
:1056C00000220C43FD0A0A3002D500200146E9E71A
:1056D0000105101969410C9C0D9D00196941FFF7E6
:1056E000A2FFDFE7F8B50546480040080C4628430E
:1056F00004D06000184A400D904201DD2846F8BDF4
:1057000015493539884210DC88420BDB290D20030E
:1057100008432903014305D0E00F1049C007411891
:105720000020F8BD00200146F8BD161A4020821B5B
:1057300028462146FFF754FF074600912846214698
:105740003246FFF71BFD3A46009BFFF76CFF3246DF
:10575000FFF746FFF8BD0000330400000000F03FF3
:10576000064C0125064E05E0E36807CC2B430C3CB4
:1057700098471034B442F7D3FFF7A6FC40B10008B5
:1057800060B1000870B58C180578401C6B075B0F82
:1057900001D10378401C2A1106D10278401C03E095
:1057A00006780E70401C491C5B1EF9D12B0705D4EE
:1057B0000023521E0DD40B70491CFAE70378401CDD
:1057C000CB1A921C03E01D780D70491C5B1C521E05
:1057D000F9D5A142D8D3002070BD000038B50446E9
:1057E000064805490068FFF783FC604300E0401E5F
:1057F00000900028FBD138BD40420F00A8010020D6
:1058000010B500231A4603E0845CE3189BB2521CD7
:105810008A42F9D3D84380B210BD000010B50348C6
:1058200000F068FB024800F065FB10BD5016002038
:105830000816002030B5446C1C252C400125A540DD
:10584000046C6560046863608368102B036803D090
:1058500099600068C26030BD9A600068C16030BD68
:1058600010B503F00BFA202003F070FF012005F0C3
:105870007FF8054804F060FF044805F069F900204E
:1058800005F070F910BD00004C000020838000007E
:1058900070B505200121000700F0F6FD0024124D2F
:1058A000124E002805D00121490330462C6000F03B
:1058B000FFF80221304600F0E7FD00280CD101225C
:1058C0008021304600F0E9FD09482C600088094934
:1058D0004000088004F0A4FC012000F00DFD02202F
:1058E00000F00AFD70BD0000A4010020000400507B
:1058F000B8000020C400002010B5082000F0FCFC17
:1059000010BD704710B5084900224A6107494B682D
:105910004C1523434B604B68082423434B60C0095C
:10592000C001026010BD0000E81700200020024006
:105930007FB500250C460646039500F01FFCE009E4
:10594000029003A901960095684600F0AFFB00287D
:1059500004D000F0E7FB002004B070BD00F0E2FBD3
:105960000120F9E710B5002302E0C45CCC545B1CB5
:105970009342FAD310BD000010B5214A002190696E
:10598000C305204804D5416902231943416191159B
:1059900093699B0505D54369012423434361630251
:1059A000194393695B0505D5436908242343436183
:1059B000E301194393691B0505D543690424234377
:1059C00043616302194393699B0405D5436910241D
:1059D000234343616302194393699B0304D54469DC
:1059E00020231C43446119439369DB0305D54369B4
:1059F000402423434361A0020143916110BD000094
:105A000000200240E817002070B5054600F04CFD6C
:105A10000646184C0AE0681C08D0002D04D000F09F
:105A200043FD801BA84201D9032070BDA069C007B7
:105A3000F1D1A069800701D50220A061A069C0054D
:105A400011D4A06980050ED4A06940050BD4A069CB
:105A5000000508D4A069800405D4A069800302D49D
:105A6000A069C00303D5FFF787FF012070BD0020A8
:105A700070BD000000200240F8B51746002605461C
:105A80000C4600F07BFB09E029460220226800F06A
:105A900057FB002804D1241D2D1D361DBE42F3D313
:105AA00000F040FBBE4201D20020F8BD0120F8BD4D
:105AB00010B500F0EEFC10BDF8B5054604464035C3
:105AC000287C0026012808D00120287420688168DD
:105AD0008907890F01290ED101E00220F8BD016874
:105AE000C90708D0606D20210843606501260020A9
:105AF00028743046F8BD616DFF22013291430222C5
:105B000011436165C1688907890F0091C1688908DF
:105B10008900C1602068816892071143816000F0AC
:105B2000C3FC07460EE000F0BFFCC01B0A2809D9E1
:105B3000606D0221884310210843606500202874AD
:105B40000120F8BD206880680028ECDB2068C1686F
:105B5000009A1143C160606D80088000401C606540
:105B6000C5E7000070B50A4D286AA91508432862E8
:105B700000F09AFC044606E000F096FC001B0328A7
:105B800001D9012070BD286A4000F5D5002070BD04
:105B900000000140F8B506460D464036317C01292B
:105BA0000DD00121317401688A68520709D5416D11
:105BB000202211434165002030740120F8BD0220ED
:105BC000F8BD174B6A68D80547109A42154C8A6A87
:105BD0002B6812D05B035B0B1A438A622968490366
:105BE00005D5A1680143A1600A20FFF7F7FD2868E9
:105BF000800312D5A06838430EE05B035B0B9A4329
:105C00008A622968490302D5A1688143A160286896
:105C1000800302D5A068B843A06000203074F8BDAE
:105C2000011000000027014070B5040006D0606D2F
:105C3000264600254036002802D006E0012070BD2F
:105C4000A5653574204600F0D3F8606DC00603D416
:105C500021688868400705D5606D1021084360659C
:105C60003574EBE7606DFF2201329043022210434E
:105C7000606588688207920F5B48012A02D10A6832
:105C8000D2072BD1032362689B079A4205D05B425F
:105C90009A4202D05B009A4209D10A6992009208A6
:105CA0000A6121680A6963681A430A610CE00A699B
:105CB000920092080A6181680F22920491438160E8
:105CC00081686268114381602168CA6818239A4319
:105CD000CA602168CA68A3681A43CA608168012241
:105CE0005206914381608168A28E52061143816001
:105CF00020688168C90004D4816801221207114319
:105D000081602068C168394A1140C1602069E1683A
:105D1000022825D000200143204620300278037B52
:105D200052035B001A431143226B1143A269920391
:105D30001143E269D20311432268D3681943D16049
:105D4000616A0A46FF3AC23A05D0A26A1143226844
:105D5000D3681943D16042780121012A02D00BE0B7
:105D60000420D8E70078002823D0606D202210435B
:105D70006065A06D0843A065E06B012820681FD016
:105D80000169C90703D00169490849000161206818
:105D90004169C908C900416120684169A26B11438A
:105DA0004161A565606D80088000401C6065002031
:105DB00070BD2068C26801231B041A43C260DBE780
:105DC0000269FF239B009A43026120680269236CE9
:105DD000A66C1A43636C33431A430261206802695C
:105DE0000A430261D3E70000002701401902FEFFC9
:105DF00010B586B0044614216846FFF7E9F90E494C
:105E00002068884216D10D48416B42151143416309
:105E1000C16A01221143C162C06A694610400590FF
:105E2000022000900320019000200290052000072E
:105E300000F06EFA06B010BD0024014000100240D0
:105E400070B50024014620314A79022A03D004218A
:105E5000C163012418E0026813680E25AB43136088
:105E6000026813685B085B001360436C1C221340DC
:105E7000012215469D40036C5D604A7100220A7143
:105E8000816B002900D08847204670BD70B50400A2
:105E900029D0206801684908490001601348256835
:105EA00014212818FFF724F980006064104820644A
:105EB00000202860626C1C210A4001239340226C60
:105EC00053600B4A8032936A656C0D400F21A940E4
:105ED0008B439362E06220636063A063E0632034DD
:105EE0006071207170BD012070BD0000F8FFFDBF22
:105EF00000000240F0B4016C0D6801680C68466C4B
:105F00001C2304221E401746B7402F420ED06707BD
:105F10000CD50C68A40602D40C6894430C60416C48
:105F200019408A40016C4A60016B1AE00227B740B1
:105F300002462F402032002F17D0A70715D50C6836
:105F4000A40605D40C680A25AC430C6001215171EC
:105F5000446C02211C40036CA14059600021117166
:105F6000C16A002918D0F0BC08470827B7402F4263
:105F700012D0240710D50C680E25AC430C60446C7D
:105F800001211C400B46A340046C6360C163517146
:105F900000211171416BE4E7F0BC704770B504005B
:105FA0003CD01F48256814212818FFF7A1F880006D
:105FB00060641C4820640221204620300246417162
:105FC00029681948E3680140A06866691843236995
:105FD00033431843A3691843E3691843236A1843FA
:105FE000084328600121A0688903884210D00D4829
:105FF0008030836A656C1C210D400F26AE40B34390
:106000008362656C63680D40816AAB400B438362B9
:106010000020E06301215171107170BD012070BD3D
:10602000F8FFFDBF000002400F80FFFFF8B50446F7
:106030008C46203001790025012909D001260671FE
:1060400041790027012905D0077102252846F8BDAE
:106050000220F8BD02214171E76320680168490808
:106060004900016061462046FFF7E4FB206B0028F1
:106070002068016801D00E2205E0042291430160EE
:10608000206801680A2211430160206801683143D9
:106090000160DBE770B5054600F006FA044600F043
:1060A00003FA001BA842FAD370BD0000F8B51A4EDF
:1060B0000546307C0F46012807D001203074174870
:1060C000FFF7A2FC010002D021E00220F8BD002071
:1060D000C04338606C6814E02046FFF713FC0F489B
:1060E000FFF792FC01460E48426808239A4342603B
:1060F000426843159A434260002901D03C6006E0A3
:106100008034A8686A68C0018018A042E4D80020E2
:1061100030740846F8BD0000E817002050C30000A6
:106120000020024005484168022211434160416855
:10613000012211434160002070470000002002400E
:10614000F8B50C4C1646207C0F46012808D00120DB
:1061500020740948FFF758FC0025002802D006E00B
:106160000220F8BD65613E600348FFF74DFC2574D1
:10617000F8BD0000E817002050C300001148416836
:10618000C9070BD0EFF3108172B60F4AC2600F4AF5
:10619000C26081F310884168C9070ED14168890740
:1061A0000DD5EFF3108172B6094A0261094A026106
:1061B00081F310884068800701D5012070470020D6
:1061C0007047000000200240EFCDAB8905040302B8
:1061D000BFAE9D8C16151413F0B500235DE00124AD
:1061E0009C4022460A4057D006685F000325BD4008
:1061F0002E43AC460660DD08AD002D182E6AAE4673
:106200005D07EF0E0F25BD40AE4375462E628668D2
:106210006546AE4386604568A5434560C4686546EB
:10622000AC43C4609D081F4CAD002D19AF689C079E
:10623000260F0F24B440A4463C4005273F07B84230
:1062400001D1002714E0184FB84201D101270FE017
:10625000164FB84201D102270AE0154FB84201D1CA
:10626000032705E0134FB84201D1052700E00627B8
:10627000B740A74210D1AE686446A643AE600E4C4C
:10628000256895432560656895436560A5689543D5
:10629000A560E5689543E5605B1C0A46DA409ED13F
:1062A000F0BD000000000140000400500008005054
:1062B000000C0050001C00500004014010B50D4CB3
:1062C000082809D002280FD0012804D103F08AFA47
:1062D0000020E071A08310BD03F084FA208D401CE3
:1062E000208502F027F910BD03F07CFA0120A0718F
:1062F00010BD0000A000002010B504494A69024208
:1063000002D04861FFF7DAFF10BD00000004014031
:10631000F8B500230124A2E027469F403A4070D000
:106320004D68022D01D0122D14D1DD08AD002D18BD
:1063300000952D6A5E07AC46F50E0F26AE46AE40C0
:106340006546B543AC460E697546AE4065462E437C
:10635000009D2E624D68012D05D0022D03D0112D18
:1063600001D0122D16D185680326AC465D00AE46DD
:10637000AE406546B543AC46CE687546AE40654610
:106380002E43866046680D79BE43ED06ED0F9D40B5
:106390003543456006685F000325BD40AE46AE4309
:1063A0000D79B446AE07B60FBE4065462E43066073
:1063B000C6687546AE438D68BD403543C5604D68BF
:1063C000ED004BD5294D6E6B26436E639E08284D1C
:1063D000B6007519AC46AD689E07360F0F27B7405B
:1063E000BD4305273F07B84201D1002715E0214FE3
:1063F000B84201D1012710E01F4FB84202D1022755
:106400000BE02BE01D4FB84201D1032705E01C4FE4
:10641000B84201D1052700E00627B7402F43654663
:10642000AF60184D2E684F689643FF0300D51643A2
:106430002E606E684F689643BF0300D516436E60AA
:10644000AE684F689643FF0200D51643AE60EE6813
:106450004F689643BF0200D51643EE605B1C0A6886
:106460001546DD4000D057E7F8BD0000001002409F
:10647000000001400004005000080050000C0050D3
:10648000001C0050000401400069084000D00120B9
:10649000704742694A4042617047002A01D08161D9
:1064A0007047816270470000014800687047000033
:1064B0007C02002002480168491C0160704700000E
:1064C0007C02002010B508480024016840221143D6
:1064D0000160204600F00AF8002801D0012401E004
:1064E00000F018F9204610BD0020024070B50546A6
:1064F00009487D210024C9000068FEF7F9FD00F07D
:106500006BFE002801D0012404E000222946501E21
:1065100000F020F9204670BDA801002070477047A8
:1065200010B503F05FF901F06BFC01F0E9FC0E49D6
:106530000120C8730D4C410300222046FFF7ADFF38
:106540000121002209032046FFF7A7FFFF210520B4
:10655000002201310007FFF7A0FF00228021204622
:10656000FFF79BFF10BD0000A000002000040050BA
:1065700070477047704710B5044600680168C9430A
:10658000C90708D18168C943C90704D10121416005
:106590002046FFF7C5FF20680168C943890708D472
:1065A0008168C943890704D4022141602046FFF76E
:1065B000B5FF20680168C943490708D48168C94309
:1065C000490704D404214160204600F0A1F8206866
:1065D0000168C943090708D48168C943090704D47D
:1065E000082141602046FFF7C3FF20680168C943C6
:1065F000C90608D48168C943C90604D41021416082
:106600002046FFF78CFF20680168C943890608D43B
:106610008168C943890604D4202141602046FFF7E0
:10662000A9FF20680168C943490608D48168C943A5
:10663000490604D4402141602046FFF79AFF10BD6F
:10664000F8B5040005D025462035A87B002802D0E7
:1066500006E00120F8BD00206873204600F040F8F5
:106660000220A8732068C26884466368012B04D0A6
:106670000120A16AC005814201D11E208243154834
:106680006169814201D0144802401448A668024062
:1066900018463043676A266A3E433043A66A304351
:1066A0001043012B03D00122D205964203D1236966
:1066B000E2681A431043074A914205D0A269114388
:1066C000E2690243084610436146C8600120A8738E
:1066D0000020F8BDFFFF00003F1FFFFFF8F119FF8A
:1066E00010B50068084988420CD10848816BC20483
:1066F00011438163002211460D2000F02BF80D207C
:1067000000F01EF810BD0000007C004000100240A8
:10671000704700000448416B012211434163816BC3
:10672000020411438163704700100240C106C90E84
:1067300001208840014908607047000080E100E0C6
:10674000C106C90E01208840014908607047000059
:1067500000E100E010B501F0E3FD10BD0248016862
:10676000821511430160704700700040F8B504467F
:106770000078544D800672D5524E0027403EB06BD3
:10678000C00004D4B06BA9050843B06301274E488C
:106790000168C90511D40168821511430160FFF732
:1067A00083FE009005E0FFF77FFE0099401A642801
:1067B00037D845480068C005F5D53268032109057A
:1067C00060680A400140914208D08103890F032983
:1067D00004D13168890301D50120F8BD2A6903215C
:1067E00009040A4022D0084090421FD02078800639
:1067F0001CD528692A6988430121C9040A432A61F2
:106800002A698A432A612861C0050FD5FFF74CFE2B
:10681000009008E0FFF748FE0099411A2B4881429A
:1068200001D90320F8BD28698005F3D56168880384
:10683000800F032805D132680005824301400A43D6
:1068400032602869032261681204114008432861FC
:10685000002F04D0B16B012000078143B163207881
:10686000C00705D0E868A168800880000843E86098
:106870002078800705D5E8680C218843E168084343
:10688000E8602078400706D5E8680321890288433C
:1068900021690843E8602078000706D5E8680321ED
:1068A0000903884361690843E8602078000606D53B
:1068B000E868032189048843A1690843E86000204F
:1068C000F8BD000040100240007000408813000036
:1068D000F8B50E4605007DD053480068C007C00FCC
:1068E000B0420AD25048016849084900314301606A
:1068F0000068C007C00FB04271D128784B4C8007A8
:1069000005D5E068F0218843A9680843E06028784D
:10691000C00752D06868022817D0032818D0216811
:10692000012818D08905002959DAE1688908890009
:106930000143E160FFF7B8FD69680746022912D0FC
:1069400003291CD0012926D033E021688903EAE716
:1069500021688901E7E74907E5E7FFF7A5FDC11BC6
:106960003348814223D8E0680007800F0228F4D121
:1069700023E0FFF799FDC11B2D48814217D8E0683D
:106980000007800F0328F4D117E0FFF78DFDC11B2E
:10699000274881420BD8E0680007800F0128F4D116
:1069A0000BE0FFF781FDC11B2148814201D9032083
:1069B000F8BDE0680007800FF3D11B480168C907E4
:1069C000C90FB1420DD9016849084900314301603E
:1069D000006800E003E0C007C00FB04201D0012012
:1069E000F8BD2878400706D5E068072109028843EA
:1069F000E9680843E0602878000707D5E0680721C8
:106A0000C90288432969C9000843E06000F036F8EC
:106A1000E168084A0906090F515CC8400649086048
:106A20000020FFF763FDF8BD002002400010024087
:106A300088130000FEAF0008A801002004480549A3
:106A40000068C968044A4905490F515CC84070474D
:106A5000A80100200010024017B0000804480549B2
:106A60000068C968044A8904490F515CC8407047EE
:106A7000A80100200010024017B0000810B5184A05
:106A8000D1680C20084004280BD0082810D00C280E
:106A900010D050680004410F0120C003491C8840F9
:106AA00010BD1068C00601D50E4810BD0E4810BDBF
:106AB0000E4810BD88020E4B000F185C0902D36807
:106AC000890F491CDB0301D5084A05E01268D2068C
:106AD00001D5044A00E0044A5043FEF709FB10BD0B
:106AE0000010024000093D000024F40000127A006A
:106AF0000EB00008FEB505007ED0FE4CE7680C2005
:106B0000E66807400120000406402878C00747D007
:106B1000082F05D00C2F0AD101200004864206D18F
:106B2000206880033CD568680028E5D038E0012063
:106B300069680004814203D121680143216011E0AA
:106B4000052301221B0492049942216802D11143BA
:106B50002160F1E7814321602168014000912068B4
:106B600090432060686800280DD0FFF79DFC0090DE
:106B700005E0FFF799FC0099401A64287AD820684C
:106B80008003F6D50CE0FFF78FFC009005E0FFF7DF
:106B90008BFC0099401A6428F0D820688003F6D452
:106BA0002878800755D50923E868042F0DD00C2FCD
:106BB00001D1002E09D000283BD021689943014320
:106BC0002160FFF771FC064627E02168490701D5DF
:106BD000002891D061681F22120291432A69120293
:106BE000114361602168994301432160FFF746FF2B
:106BF000E16809060A0F00E079E1BF49895CC840F5
:106C0000BE4908600020FFF771FC002872D120E027
:106C1000FFF74AFC801B0228B0D820684007F7D550
:106C200060681F21090288432969090208436060DE
:106C30000FE02068400840002060FFF735FC064662
:106C400004E0FFF731FC801B022897D8206840073A
:106C5000F7D42878C0065FD5002F0CD0A86900288B
:106C600049D02068FF21013108432060FFF71CFC58
:106C700006462DE0C0E02068800502D5A8690028FE
:106C8000A7D06068072149038843296A08436060E8
:106C90006068297F0002000A090608436060286ACC
:106CA000410B0120C003491C8840E16809060A0F16
:106CB0009149895CC840914908600020FFF716FCA3
:106CC000002817D128E0FFF7EFFB801B0228A3D88C
:106CD00020688005F7D56068072149038843296A41
:106CE000084360606068297F0002000A09060843C3
:106CF000606011E0E1E02168FF2001308143216004
:106D0000FFF7D2FB064604E0FFF7CEFB801B02280C
:106D100072D820688005F7D42878794E000724D5EA
:106D200068690028306910D0012108433061FFF7FD
:106D3000BBFB009005E0FFF7B7FB0099401A022863
:106D40005AD830698007F6D50FE04008400030611E
:106D5000FFF7AAFB009005E0FFF7A6FB0099401A99
:106D6000022849D830698007F6D42878400765D5CD
:106D700000200290A06BC00006D4A06B012109077F
:106D80000843A063012002905E480168C90511D440
:106D90000168821511430160FFF786FB009005E052
:106DA000FFF782FB0099401A642825D855480068EF
:106DB000C005F5D5FF20AA680130824203D13169B0
:106DC0000143316111E001218902002A07D0052326
:106DD0001B029A4203D132690A433261EFE73269FA
:106DE00082433261306988433061A86800280FD03F
:106DF000FFF75AFB009007E05EE0FFF755FB0099B4
:106E0000411A4148814257D830698005F5D50DE0D7
:106E1000FFF74AFB009006E0FFF746FB0099411A96
:106E20003948814248D830698005F5D40298002855
:106E300004D0A06B012109078843A063686A002879
:106E400064D00C2F3ED0012636060228206805D0DB
:106E5000B0432060FFF728FB05462FE0B0432060D9
:106E6000FFF722FB074604E0FFF71EFBC01B0228CA
:106E700022D820688001F7D4E96AA86AE26808434A
:106E8000296BFD231B049A4311430843E0602068EB
:106E900030432060FFF708FB054604E0FFF704FBE2
:106EA000401B022808D820688001F7D52EE0FFF7A4
:106EB000FBFA401B022801D90320FEBD2068800197
:106EC000F5D423E00128F8D0E06801210904AA6A7A
:106ED000014091420BD10F218904EA6A014091429D
:106EE00005D1032189050840296B88420ED0012075
:106EF000FEBD000000100240FEAF0008A801002007
:106F00004010024000700040881300000020EFE7AE
:106F100070B5040007D0002625464035A662687C7F
:106F2000002802D005E0012070BD2E74204600F03C
:106F30002FF80220687420680168402291430160A4
:106F4000A168606822690843E168114308436169E8
:106F500001220843A169520211400843E169084334
:106F6000216A0843A16A084321680860A0690421D6
:106F7000000C0840616A0843216848602068C169C4
:106F800092009143C161666501206874002070BD64
:106F900010B586B0044614216846FEF719F9104969
:106FA0002068884219D10F48416B82141143416314
:106FB000C16A01221143C162C06A002110400590DC
:106FC000E0200090022001900320039002910491A0
:106FD000052069460007FFF79BF906B010BD0000C9
:106FE0000030014000100240FFB5044683B001208C
:106FF00001900020264640360090307C0C9F1D46B4
:1070000001280FD001203074FFF74EFA0290707CF7
:10701000616801280DD0CA1FFD3A08D1A168002976
:1070200005D102E0022007B0F0BD042801D0022003
:10703000C3E00498002828D00598002825D0002D0A
:1070400023D0707C042801D0052070740020606576
:107050000599A163E587A58704992163E586A5863F
:107060002064606420680168490603D401684022F6
:10707000114301600121E068C9028842606848D17B
:10708000002804D0012D02D03CE0012095E0206BC7
:1070900021680088C860206B801C2063E08E401E41
:1070A000E0862FE020688168890710D5E18E0029ED
:1070B0000DD0019901290AD1216B0988C160206B8B
:1070C000801C2063E08E401EE08600200190206836
:1070D0008168C9070DD0E18F00290AD0C068A16B73
:1070E0000880A06B801CA063E08F401EE087012019
:1070F0000190FFF7D9F901460298081AB84201D366
:10710000781C59D1E08E0028CCD1E08F0028C9D15D
:1071100046E0002801D0012D3CD1206B2168007889
:107120000873206B401C2063E08E401EE08631E037
:1071300020688168890710D5E18E00290DD001995A
:1071400001290AD1216B09780173206B401C20634F
:10715000E08E401EE0860020019020688168C9070B
:107160000DD0E18F00290AD0C068A16B0870A06B18
:10717000401CA063E08F401EE08701200190FFF7D4
:1071800093F90299401AB84202D3781C02D013E056
:10719000002F11D0E08E0028CAD1E08F0028C7D17F
:1071A00039462046029A01F091FD002807D00120BF
:1071B00000902020606509E00320009006E0A068B0
:1071C000002803D12068C168806801900120707494
:1071D00000203074009826E7094910B5401E884207
:1071E00001D9012010BD074C60610321081F01F087
:1071F00097F80020A06107202061002010BD00004A
:10720000FFFFFF0000E000E0F0B502462032137EF1
:10721000012B15D0012717760223537605686C6879
:10722000AB687026B4430E68496826438024A343A4
:1072300019436E6000688160577600201076F0BDBB
:107240000220F0BD10B586B0044614216846FDF753
:10725000BFFF012120688907884214D10B48C16A09
:1072600001221143C162C06A02211040059008202A
:10727000009000200290039001910491052069463E
:107280000007FFF745F806B010BD000000100240EF
:10729000F8B5064604462036307E0D4601280DD04E
:1072A00001203076022070760427002A08D0042AB4
:1072B00016D0082A2AD00C2A4DD137E00220F8BD7A
:1072C000206802F035FB2068816908221143816142
:1072D00020688169B943816120688169EA6812E0A8
:1072E000206802F03DFB206882690121C9020A433F
:1072F0008261206881690122920291438161206844
:107300008169EA6812021143816124E0206802F079
:1073100040FB2068C26908210A43C2612068C16934
:10732000B943C1612068C169EA6812E0206802F0CF
:107330004BFB2068C1690122D2021143C161206860
:10734000C269012189028A43C2612068C169EA6871
:1073500012021143C1610120707600203076F8BD21
:1073600070B5040005D025462035687E002802D07F
:1073700006E0012070BD00202876204600F00AF8C3
:1073800002206876211D206802F0A6FA01206876A6
:10739000002070BD006801218907884204D103489C
:1073A000816B01221143816370470000001002408D
:1073B00010B502F017FA01200349024608730A319A
:1073C000024800F00FFA10BDA0000020AC1300200E
:1073D00070B5040017D02420606720680168490850
:1073E000490001602068002505602068456020682C
:1073F0008560204600F0DEF8E5676567A5676034C4
:107400002574002070BD012070BD7047F8B502687A
:107410000446D0691168936805072D0F5BD0DD071E
:10742000ED0FFF2621360E402E4367D0C60706D04B
:10743000CE0504D501261662E26F3243E267870764
:1074400002220426002F06DADF0704D027683A62FA
:10745000E76F3743E767470706D5DB0704D02368A4
:107460001E62E36F1343E367020709D520220A4037
:107470002A4305D0236808221A62E36F1343E367A7
:10748000E26F002A2FD0800606D5880604D5216E2B
:10749000002901D020468847E06F216889684906A5
:1074A00001D4000724D5204602F058FC20688168EA
:1074B000490619D58168402291438160E06E002819
:1074C00012D020498163E06EFEF7BAFC00280AD092
:1074D000E06E816B06E0850610D58D060ED5216E17
:1074E0001CE020468847F8BD2046FFF78EFFF8BD18
:1074F0002046FFF78AFF0020E067F8BDC50208D5E7
:107500005B0206D50120000510622046FFF750FF00
:10751000F8BD030605D50B0603D5616E0029E0D141
:10752000F8BD4006FCD54806FAD513682046402130
:107530008B431360202161670021616600F05EFAD1
:10754000F8BD0000B99C000810B5040003D0606FBE
:10755000002802D007E0012010BD00217020015555
:10756000204600F05BF82420606720680168490825
:1075700049000160204602F093FC0128ECD0606ACB
:10758000002802D0204602F07BFA206841680922D8
:10759000D20291434160206881682A229143816030
:1075A00020680168012211430160204602F0CEFAF2
:1075B00010BD000010B50446144A016814489142F9
:1075C0000BD1816B012292049143816303218902D3
:1075D0001048FEF701FE1D2014E00F4A914213D11E
:1075E000416B01229203914341630321052049022B
:1075F0000007FEF7F1FDE06EFEF748FCA06EFEF717
:1076000045FC1B20FFF792F810BD00000048004029
:10761000001002400004005000380140F0B587B06F
:10762000054614216846FDF7D3FD394F2B683948CC
:107630000222042100240326BB4218D1836B0D04CF
:107640002B438363C36A1343C362C06A049110402F
:107650000590B0026B4655C369462F48FEF758FEA9
:10766000002211461D20FFF775F81D204CE02B4F1E
:10767000BB424BD1436B0127BF033B434363C36A08
:1076800001273B43C362C06A049138400590032040
:1076900040026B4655C3052069460007FEF738FED9
:1076A000204F1F48BC60FC6041C7FC6080203C61EB
:1076B000B860202078610002B8611A48083FFEF7E0
:1076C0006DFC002801D0FEF71CF9EF661448BD627E
:1076D000154F143841C710207C603860FC603C6155
:1076E0007C618020BC61B8600F48083FFEF756FC03
:1076F000002801D0FEF705F9AF66002201211B200A
:10770000BD62FFF727F81B20FFF71AF807B0F0BD9E
:1077100000480040001002400004005000380140C2
:10772000300002400816002050160020F8B504462C
:10773000806F20284DD100290BD0002A09D00123C9
:10774000A0681B03984206D12069002803D1C8070E
:1077500001D00120F8BD25466035287C012838D0AD
:10776000012028745820616502530026E667222014
:10777000A067E06E002819D01749C162E16E174872
:107780000863E16E16484863E06E13468663676DD2
:1077900021683A462431E06EFEF748FC002805D007
:1077A0001020E0672E7420206067D2E72E742068D6
:1077B0000168FF22013211430160206881680122C3
:1077C000114381602068816840221143816000205C
:1077D000F8BD0220F8BD0000159D0008539D00086B
:1077E000CD9C0008F0B5836F202B54D100290AD01E
:1077F000002A08D08568DC01A54206D10369002B68
:1078000003D1CB0701D00120F0BD034660331E7CBD
:10781000012E40D001261E744165014640310A8385
:107820004A830022FF260266A54204D10569002D85
:1078300013D11A4D0AE07F27002D09D00126360703
:10784000B5420CD10569002D05D03F258D8307E099
:107850000569002D01D08F8302E08E8300E08A83CA
:10786000C2672221816701688D68012635438D60DA
:107870008168A14202D1016900290AD00849016644
:107880001A7400680168FF22213211430160002050
:10789000F0BD0449F3E70220F0BD0000FF01000045
:1078A000499E0008F19D000870B51C481B4C0278E9
:1078B0000A3C1B48617B4254491CCAB2801862735F
:1078C0002038C17F0A2923D1807F0D2820D120466E
:1078D00013493C30FDF763FC657BA573C821104854
:1078E000FDF776FC0020607320730120E072607861
:1078F000282D06D900280BD10122110205200007EE
:1079000004E0002804D1012280210648FEF7C5FDCD
:10791000012202490448FFF765FF70BDAA0000205C
:107920004015002000040050AC1300207047FFB544
:107930000446406F83B017460D4620285CD1002DC9
:107940000AD0002F08D0A168C001814207D1206968
:10795000002804D1E80702D0012007B0F0BD20467E
:1079600060300290007C012846D002980121017409
:107970000020E06721206067FEF796FD264640362E
:107980000190378277820120A1680003814202D1F1
:107990002069002802D02F46002511E000270FE0C3
:1079A00000228021204602F08FFB002815D1002FF5
:1079B00015D02168387888627F1C708A401E7082DA
:1079C000708A019B002806980090E9D1002240218E
:1079D000204602F079FB002808D00320BDE7288864
:1079E0002168C005C00D8862AD1CE6E720206067F5
:1079F000029900200874B0E70220AEE7704700004B
:107A000001490248C160FDE70400FA0500ED00E00D
:107A100070B501240E4D6402002221462846FEF76F
:107A20003CFD002261102846FEF737FD0A2002F0D7
:107A300012FE012221462846FEF72FFD0A2002F001
:107A40000AFE002221462846FEF727FD70BD0000F1
:107A50000004005070B501240E4D6402002221463E
:107A60002846FEF71AFD012211022846FEF715FDF1
:107A70000A2002F0F0FD012221462846FEF70DFD06
:107A80000A2002F0E8FD002221462846FEF705FD07
:107A900070BD000000040050F1B500240126164F0F
:107AA00025467602002231463846FEF7F6FC0A20CB
:107AB00002F0D1FD012231463846FEF7EEFC6006A9
:107AC000040EFF2101313846FEF7DEFC002801D00C
:107AD000641CE4B2052002F0BEFD6D1CEDB2082D61
:107AE000E0D30098002803D0FFF792FF2046F8BDAE
:107AF000FFF7B0FFFAE7000000040050F8B50126D8
:107B0000164F05467602002231463846FEF7C5FC80
:107B10000024E80901D0012200E00022FF21013108
:107B20003846FEF7BAFC6806050E0A2002F093FDFF
:107B3000012231463846FEF7B0FC0A2002F08BFDE8
:107B4000002231463846FEF7A8FC0A2002F083FDE9
:107B5000641CE4B2082CDCD3F8BD00000004005023
:107B600070B501220C4D140221462846FEF795FC03
:107B70000122560231462846FEF78FFC002221469C
:107B80002846FEF78AFC0A2002F065FD00223146F5
:107B90002846FEF782FC70BD0004005070B5012439
:107BA0000E4D6402002221462846FEF776FC661040
:107BB000002231462846FEF770FC0A2002F04BFDF9
:107BC000012221462846FEF768FC0122314628465C
:107BD000FEF763FC0A2002F03EFD70BD0004005079
:107BE000F8B50122144D1602002431462846FEF74E
:107BF00054FC062002F02FFD012257023946284688
:107C0000FEF74BFC062002F026FD07E0641CE4B200
:107C1000FA2C03D9FFF7C2FF0120F8BD31462846F0
:107C2000FEF732FC0028F1D1002239462846FEF743
:107C300034FC0020F8BD000000040050F8B5204ED0
:107C400040213046FEF720FCFF27002501371D4C60
:107C500000282DD001F0AAFF01F0E2FF1A480560CC
:107C60006078002803D10120607002F0D9FA2078F2
:107C7000632806D9002280213046FEF70EFC01223F
:107C800005E0012280213046FEF707FC16E00520C2
:107C900039460007FEF701FC0C480D4A0188914265
:107CA00002D1C088002802D10B490A48C860F8BD3B
:107CB0006078012802D1657002F08AFA0022E6E7B6
:107CC00000040050A0000020A4010020800B002030
:107CD000AA5500000400FA0500ED00E010B51848B0
:107CE00000F032F81648401E41788170372120207C
:107CF00000F071F80321212000F06DF840212220CE
:107D000000F069F80821232000F065F8AA2130204E
:107D100000F061F80B4802210187322000F05BF887
:107D20000121332000F057F85F21202000F053F8A4
:107D3000034800F009F80A2002F08DFC10BD000095
:107D400001000020800B002010B501460F2000F03C
:107D500021F8002800D0012010BD10B50446FFF71F
:107D6000FFFE3220FFF7CAFEFFF73AFFE0B2FFF74F
:107D7000C5FEFFF735FFFFF7F3FE3320FFF7BEFE2A
:107D8000FFF72EFF0020FFF787FE0446FFF706FFF0
:107D9000204610BD10B50C46FFF7DFFF2070012014
:107DA00010BD70B50D460446FFF7DAFE3220FFF72E
:107DB000A5FEFFF715FFE0B2FFF7A0FEFFF710FFEB
:107DC0002846FFF79BFEFFF70BFFFFF7E7FE0A20B1
:107DD00002F041FC70BD10B5FFF7E3FF012010BDBC
:107DE00010B50248FEF7C7FB10BD00007C13002051
:107DF00010B50248FFF70AFB10BD0000AC130020CD
:107E000010B50D480078002805D001220520110288
:107E10000007FEF742FB094C40212046FEF734FBE9
:107E2000002808D1064800780F2804D20122110347
:107E30002046FEF732FB10BD6B000020000400500E
:107E4000A000002070B500F03BF8194C0020A07392
:107E5000184D07212A7DE08B01F082FC1648332162
:107E600001700E2141703638A98801872246128C94
:107E7000428701462A46233093780376D2784276A9
:107E8000821E28462230037D1377437D53772231AB
:107E9000808A88830E210848FDF7B2FC0649608479
:107EA0000A31888005481021826A0348904770BDD6
:107EB00060000020800B00205612002020B0000837
:107EC0000D48002301784A1CD2B202700B481E29CB
:107ED00002D90121417300E043730178002903D0E6
:107EE000032A00D9037070470021C9430184FF2190
:107EF000C331C18370470000780200206000002079
:107F0000F8B53B4C1021615E481C2082002901DD40
:107F100001F076FDFFF7D4FF0025A573354E07214C
:107F2000327DE08B01F01CFC608A411C6182E12102
:107F30000901884202D92078012852D02E4D2220F2
:107F40002870E07A2E4F80001E3068702846363840
:107F5000B1880187014626480646008C4887207B69
:107F6000A871401C2073254820360078E871022152
:107F70003846FEF789FA002837D0002021490978D1
:107F80004900084328721C48317913380177717908
:107F90004177E07A1849E872420064390846703047
:107FA000FDF7FDF8E07A144942005019C8390C3049
:107FB000FDF7F5F8E07A81000F480C31FDF720FC61
:107FC0006084E17A89004A1990810F480E31826AF3
:107FD000C9B209489047012251033846FEF75DFABD
:107FE000F8BD6582FFF72EFFF8BD0120C6E700004F
:107FF00060000020800B002056120020A00000200E
:1080000000040050A700002020B000081CB500218B
:1080100017480091154A01910260C1631205816001
:1080200042608163012202610246C1602032117008
:10803000FF235170C2334362816211730163816116
:10804000042241634261C161FDF7EEFD09480090E1
:1080500001200003019069460548FDF79BFDFDF7EF
:1080600081FD00210248FDF727FD1CBD00240140D1
:10807000201300200000024408B50848016B0122CB
:1080800011430163006B01211040009000220A207F
:10809000FEF760FB0A20FEF753FB08BD001002400C
:1080A000F0B587B014216846FDF792F85148C16ACF
:1080B00004273943C162C16A39400591C26A8021EF
:1080C0000A43C262C26A0A400592C16A0125294375
:1080D000C162C16A29400591C16A02263143C16269
:1080E000C06AFF21304005900520002205310007BD
:1080F000FEF7D3F90520012210210007FEF7CDF984
:1081000001223D493D48FEF7C8F900223C493B4861
:10811000FEF7C3F93B4800903B480190002405203E
:10812000694602940007FEF7F3F8FF20053000903F
:10813000052002946946019503940007FEF7E8F8CC
:1081400010200090052069460396019502940007CF
:10815000FEF7DEF811200190029469460095039421
:108160002648FEF7D5F82948019069460096029501
:108170002248FEF7CDF80194694620480097029402
:10818000FEF7C6F81E4800900294694601950394D4
:108190001A48FEF7BDF8082000901B480190694678
:1081A00002941648FEF7B4F840206A4651C2694668
:1081B0001248FEF7ADF80320000200901120019054
:1081C00003200390029469460C48FEF7A1F80022B0
:1081D00002210520FEF7BEFA0520FEF7B1FA0022C3
:1081E00001210620FEF7B6FA0620FEF7A9FA07B02D
:1081F000F0BD000000100240010300000004005028
:10820000B07000000180000000001110000021107B
:1082100010B50F4C0D482060FF2005306060002035
:10822000A060E06020616061E0610121206249029C
:108230006062A161A0620720E0622046FEF768FE4E
:108240002068016840221143016010BD00300140E8
:10825000AC14002010B586B0002405940121134809
:1082600004940094019402948907039401601F21EF
:10827000846041600461F9214461C160FFF770F8D6
:10828000049404A909480594FEF7BEFF60200090FD
:10829000019402940C22694603940448FEF7F8FF07
:1082A0000248FEF7CFFF06B010BD00000415002005
:1082B00000B585B014216846FCF78AFF16481549B9
:1082C0000160E1214902416000218160C1600161DA
:1082D00081610C22C1614261016230214162012150
:1082E000090381634900C163FFF72EF90120800271
:1082F00000900220019001200290032003900420AE
:108300000490052069460007FEF702F801F05AFFC5
:1083100005B000BD003801402C140020704700005B
:108320008307FF22DB0E9A408907090E9940002837
:108330000BDA0007000F0838830808489B0018185C
:10834000C36993430B43C3617047830804489B0090
:108350001B181868904308431860704700ED00E050
:1083600000E400E070470000F0B5404985B03E48A9
:10837000086002F053FD3E4800F00FFD3D4CE083E5
:108380003B48801C00F009FD20843948001D00F0A6
:1083900004FD6084FF20384D01306880052068812D
:1083A000E9887D27FF00B94200D2EF803249334A85
:1083B0004031097921720491E98EC9B2117003919B
:1083C0000021E9872171A98F6171E070A88802906E
:1083D00020632889FDF7C4F80222FDF797F802F020
:1083E000CFF80022264BFCF7FFFEFDF7C7F886B258
:1083F0006682E888019031460090FCF779FEA08201
:1084000001460298FCF774FE71438EB27D20C000D5
:1084100026827043FDF7A4F81A4A1B4BFCF7FEFFB7
:10842000FDF7ACF8E082668338460099FCF760FE01
:108430002083688F60720499002903D10120207184
:108440000A2060720198002800D1EF8003990B4840
:10845000432901D943210170962207490B48FCF7B3
:108460009EFE05B0F0BD00004DA2000844000020B3
:10847000004F0008A0000020800B00200A00002010
:1084800000000840F853E3A59B843E40AC0C00205C
:108490000120704710B500280DD00A4A0021CB00FA
:1084A000D458844209D89B189B68834205D9C800D8
:1084B0008018007B10BD1F2010BD491CC9B21529B2
:1084C000EDD3FEE790B0000810B500F0C9FC03281A
:1084D00004D0042803D0052803D0002010BD0220BA
:1084E00010BD012010BD03207047000010B50E4CD8
:1084F00020610E4800F044FD002000F0A5FF01209F
:1085000000F01DFF0021084600F0F2FD04210020CC
:1085100000F0D6FF064800231A46014600F029FE67
:108520000020A07010BD0000B001002041860008AE
:10853000FFFF0000F8B508213448FDF7A5FF01282A
:1085400062D1334C0020A07000F080FC0546314819
:1085500000F072FCE80706D02069002803D000680C
:10856000002800D08047A80718D5FF2269462A486E
:1085700000F0C2FC2848143800F07AFC206900287A
:108580000CD08668002E09D023480D2314380C2205
:10859000C3568256684601781F48B047680606D51C
:1085A0002069002803D00069002800D080472806F1
:1085B0000AD52069002807D08169002904D0E84342
:1085C000C005C017401C8847A80514D500F048FC1A
:1085D000042804D000F044FC052805D00BE02069F5
:1085E000002808D0406803E02069002803D0C06854
:1085F000002800D08047A80606D52069002803D0AF
:10860000C068002800D08047F8BD0000000400507A
:10861000B0010020FFFF0000AC16002070B50C4632
:10862000012500F0A5F8204600F090FE002000F0A3
:1086300033F80120FDF72EFD00F03CFA284670BD0E
:108640000149012088707047B001002070B50025F5
:10865000012000F08DF8002000F0A4FE002401208D
:10866000FDF718FD00F05EFCC007C00FA040641CC1
:108670000543E4B2202CF2D300F01CFA284670BD6A
:1086800010B500F0DFFC10BD10B500F0E3FC10BD2C
:1086900010B500F047FC10BD10B5044600231A4683
:1086A0000649074800F065FD06484078002801D0DB
:1086B000054800E0A00100F075FE10BD02020000B8
:1086C000FFFF0000B0010020FFFFFF0010B50446CF
:1086D000074800231A46014600F04BFD0548407844
:1086E000002801D0044800E0A00100F06DFE10BD9C
:1086F000FFFF0000B0010020FFFFFF0070B505463E
:108700000C480C4600231A46014600F032FD00F0EA
:10871000EDFB01460848012909D00472064800F023
:108720009FFD00222146284600F0DAFC70BDC4738C
:10873000F4E7000001020000AC17002010B500F0C3
:1087400005FE10BD10B5084B084A012808D0D079A5
:10875000012804D119701172044800F081FD10BD88
:108760001970D173F8E70000B0010020AC170020A9
:1087700010B50A4C012805D0002000F0CBFD0020E8
:10878000607010BD012000F0C5FD61782078814245
:10879000F7D0607000F004F810BD0000B3010020B5
:1087A00070B504460B48047044700120FFF7E0FFE9
:1087B0001D208001451C002C04D0342100F048FF0E
:1087C000442103E0142100F043FF2421284600F057
:1087D0003FFF70BDB3010020FFB587B01646594971
:1087E000199A119F149B4A701399002902D0554978
:1087F0000B7002E05349FF220A70534C0146204699
:108800002830254620350190002918D001296ED145
:10881000002000F02BFE1298C0B200F0BEFC012335
:108820002B72F0B22876494A0899515C69760A9908
:10883000A976089900295CD001295CD05DE0002070
:1088400000F014FE002028720B20E66228750898BC
:10885000FFF720FE687500202070F800608004207B
:108860002071182060710020A071139901204140EF
:10887000344FE171397821721599002900D0F22026
:1088800060720020A07200F0DFFD287A002800D07E
:108890000120FFF76DFF019800F086FC2A4800F0E8
:1088A000DFFC2BA003C80490059104A800F0E5FDAF
:1088B000294800F045FE3046FCF752FE02460B46C2
:1088C00000202649FCF7AAFD0322FCF71FFE044600
:1088D0000D461298FCF744FE22462B46FCF736FD67
:1088E00000221F4BFCF732FDFCF748FEF8600BB08E
:1088F000F0BD0B2E09D00C2E07D00021E976237095
:10890000052804D0062802D006E01946F6E70C2F09
:1089100002D20C20A08100E0A7811398094DA0731A
:108920002878E07315982074189860740120FFF778
:108930001FFF019800F038FC034800F091FC094843
:10894000E860D4E7B0010020AC1700208CB000082C
:10895000C194C10000000000FF0100000000F03FD2
:1089600000408F40FFFF000010B500F047FD10BD34
:10897000FFB5454D83B00246294628312C460E9E50
:108980000C9820340291002A02D0012A73D138E0D9
:1089900000272772E8620B2020751846FFF77AFD42
:1089A0006075059828632F70F00068800420287196
:1089B00018206871AF710F9901204140E971109939
:1089C000002902D0F221697200E06872A8720020CA
:1089D00000F03AFD207A002800D00120FFF7C8FE01
:1089E000029800F0E1FB284800F03AFC27A103C9F7
:1089F00000900191684600F040FD264800F0A0FD7F
:108A000039E001212172C2B2234F2276FF5C6776E2
:108A10000D9FA776002B02D0012B02D003E00B287C
:108A200009D00C2807D00020E0762970052A04D050
:108A3000062A02D006E0E176F7E70C2E02D20C20DF
:108A4000A88100E0AE810F98A87314480078E873FD
:108A50001098287413986874002000F0F5FC207AB0
:108A6000002800D00120FFF783FE029800F09CFB55
:108A7000054800F0F5FB049800F08EFC07491498B7
:108A8000886007B0F0BD0000AC170020C194C100A1
:108A900000000000FF0100008CB00008B0010020C1
:108AA00010B50C4600F052FC204600F075FC00F0BA
:108AB000FFFC10BD08B5002069460090087804212D
:108AC000084369460870009800F0B0FC0220FDF7EA
:108AD000E1FA08BD10B5002000F0B6FC10BD10B5DD
:108AE00000F010FB10BD0000F3B50246002057490E
:108AF0008BB0002A56D0012A7DD10F462037787ED0
:108B000030225043524A3C7E80180C22121BD20065
:108B10008018C21FF93A1046466C0846156C8089C9
:108B2000FCF71EFD00224B4BFCF75EFB2A4633464A
:108B3000FCF70CFC07910690B87E8007800F001DA3
:108B4000FCF70EFD05910490F87E002800D002206D
:108B5000201A8000FCF7F0FC07460C980391C00037
:108B6000A100411A3948027C807B12018918012832
:108B700052D00020081A1C30FCF7DEFC3A46039B5A
:108B8000FCF74CFC01F0FCFC059B049AFCF7DEFBB7
:108B9000002207460C461346FCF70EFD3ED238462F
:108BA00021463DE00C46C86AFCF7DAFC06460F4653
:108BB0000C98FCF7D5FC0D46069061796088C908D1
:108BC0004018FCF7CDFCE279002A1ED00022224B8F
:108BD000FCF70AFB2B46069AFCF706FB627A022A90
:108BE00016D000221346FCF7FFFA0322FCF78EFC96
:108BF00032463B4600E027E0FCF710FC0022174B12
:108C0000FCF7A4FB02F06EF91CE000221346DFE73C
:108C1000002201239B07E6E71420ABE70020014672
:108C200000220F4BFCF7E0FA2A463346FCF78EFB96
:108C3000079B069AFCF7D8FA0A4A0B4BFCF7D4FAC2
:108C400002F03EF8FCF79AFC0DB0F0BDAC17002026
:108C5000C8010020000011400000F03F00408F409C
:108C6000000020402B8716D9CEF7EF3F10B500F05B
:108C7000EFFC10BD10B500F0F1FC10BD70B586B072
:108C800014216846FCF7A4FA01250F4EAD0300221B
:108C900029463046FDF701FC012000240190029492
:108CA0006946009503943046FDF732FB032001909E
:108CB00002946946009503943046FDF729FB022093
:108CC00001F0C2FC06B070BD0004005038B5044687
:108CD0004068FF2305332025984204D100920B46BB
:108CE0000022802107E05120005D05280DD100926F
:108CF0000B4600220121204600F009F8002804D08C
:108D0000606D28436065032038BD002038BDF8B58C
:108D10001D4617460E46044609E0681C07D0FDF7BD
:108D2000C3FB0699401AA8420BD2002D09D0206837
:108D30008168304688432ED00020B842EDD1002013
:108D4000F8BD20684168E022914341606068C11F1E
:108D5000FD390CD10121A068C903884202D0491114
:108D6000884204D1206801684022914301600120BB
:108D7000A16A4003814207D121680A6882430A60E0
:108D800021680A6802430A600120403460740020B0
:108D900020740320F8BD0120CFE70088704770479A
:108DA00070477047174908B5884204D9E1216846E1
:108DB0000170E9211EE01449884204D9D721684690
:108DC0000170D82116E01149884204D9C1216846B2
:108DD0000170C5210EE00E49884204D9752168460C
:108DE0000170812106E00B49884204D96B21684655
:108DF00001706F21417002226946982000F004FC46
:108E000008BD000000E9A43580F8A9328044E52DB2
:108E1000000B6B1B40FC541910B506484078002825
:108E200001D0062803D100F0B1FBFFF7BAFF00F034
:108E3000A1FB10BD5802002008B5020A69460A705D
:108E400048700222104600F0DFFB08BD08B5022280
:108E50006946122000F0D0F86846008840BA08BD84
:108E600001484078704700005802002002207047F7
:108E700038B5044603226946142000F0BDF81A49AB
:108E800088782070002808D0012816D014212046A8
:108E9000FCF79EF90F20207038BD684600782071DD
:108EA0006846407840424010A07168468078404251
:108EB000401060710020A06038BD684600784042D4
:108EC0004010207368464078802801D2800802E074
:108ED000FF38013880106073684680784042401047
:108EE000A0734868206138BD58020020014880788E
:108EF0007047000058020020F8B50C4606460020D6
:108F0000694608701546204600F018F82278AA42F3
:108F100001D90120F8BD68463146007800F042F8DA
:108F20000020F8BD08B501226946152000F064F85C
:108F3000684600784042401040B208BD38B50D4642
:108F4000044602226946132000F056F80A48807849
:108F5000012809D1094800F075F8C00904D0074874
:108F6000801E00F06FF801E06846007820706846C7
:108F70004078287038BD0000580200200407000027
:108F800010B500F093F800F001FB002000F05CFA4F
:108F9000012000F0E7F802490120487010BD0000F0
:108FA00058020020F8B515460E460446FFF734FF78
:108FB000104F002220213846FDF76FFA1E2000F0E6
:108FC000B1FB204600F0AEFB002000F0ABFB00241C
:108FD00005E0002000F0A6FB3055641CA4B2AC42B2
:108FE000F7D3012220213846FDF757FA00F0C2FAE4
:108FF000F8BD000000040050F8B515460E460446C2
:10900000FFF70AFF0E4F002220213846FDF745FAF0
:10901000204600F087FB002000F084FB002405E0E0
:10902000002000F07FFB3055641CA4B2AC42F7D3A3
:10903000012220213846FDF730FA00F09BFAF8BDF6
:109040000004005008B50122694600F003F86846A4
:10905000007808BDF8B515460E460446FFF7DCFE5D
:10906000114F002220213846FDF717FA1D2000F08D
:1090700059FB200A00F056FBE0B200F053FB002041
:1090800000F050FB002405E0002000F04BFB3055C1
:10909000641CA4B2AC42F7D3012220213846FDF76C
:1090A000FCF900F067FAF8BD0004005010B50A2082
:1090B000FCF7F0FF094C002210212046FDF7EDF9E6
:1090C0007D20000101F0C7FA012210212046FDF7A2
:1090D000E4F90A20FCF7DEFF10BD00000004005098
:1090E00010B5144600F024F9204600F0CFF910BD69
:1090F00008B56A4610705170022269468F2000F050
:1091000083FA08BD10B500221146C52000F07CFA94
:1091100001490720487010BD5802002008B5020A16
:1091200069460A70487004488078002803D10222FA
:10913000024800F093FA08BD58020020BE06000065
:1091400008B5020A69460A70487004488078002809
:1091500003D10222024800F081FA08BD5802002023
:10916000BC06000001B5012269469D2000F04CFAC2
:1091700008BD7CB5050A6C4625706070080AA070B1
:10918000E170100A20716271180AA0710822E3715F
:109190006946104600F038FA7CBD01B501226946E7
:1091A000A02000F031FA08BD7CB5044600200090F4
:1091B0000190224920788978884201D000F0AAF8ED
:1091C0002078002810D001280DD1217C684601703C
:1091D000617C4170A17C8170E17CC1700422694690
:1091E0008B2000F011FA7CBD08256068FCF7B8F907
:1091F00002460B4600201249FCF710F90522FCF745
:1092000085F9FCF7BBF9020C69460A70020A4A703C
:109210008870207BC870607B0871A068FCF7A0F99B
:109220000022084BFCF7FAF8FCF7A8F9020C694693
:109230004A71020A8A71C8712A46D1E75802002091
:1092400080847E418084EE3F38B56C46207061702A
:10925000A270E37004226946952000F0D5F938BD6C
:109260003EB50446002000900190029024492078E9
:109270008978884201D000F04DF82078002814D079
:10928000012811D1A18906220B0A6846037041709A
:10929000A17B8170E17BC170217C0171617C417196
:1092A00069468C2000F0B0F93EBD607AF12802D00A
:1092B000F22808D00EE01348FFF742FF1248FFF7EC
:1092C0002DFF022006E01148FFF73AFF1048FFF794
:1092D00025FF0620618809220B0A69460B70A378D6
:1092E0004B7023798B706379CB70A3790B71E37921
:1092F0004B71237A8B71C871A07A0872D0E7000095
:1093000058020020FFFF0000058000000F1D000034
:109310002110000001B568460449007888700122D8
:1093200069468A2000F070F908BD0000580200204C
:109330000A4610B50146002000F040F910BD01B505
:1093400001226946962000F05FF908BD38B5104C3F
:1093500005462078002804D12846FFF723FD012088
:1093600020702846FCF7FCF800220A4BFCF756F860
:10937000FCF704F9020E69460A70020C4A70020AF0
:109380008A70C8700422862000F03EF938BD0000C3
:10939000580200208084EE3F10B5022100F090F8C2
:1093A00010BD000008B5074A05215170020C69463E
:1093B0000A70020A4A7088700322822000F024F9A1
:1093C00008BD00005802002038B5044609490520B0
:1093D00048709621084800F03BF9210C684601705E
:1093E000210A4170847003226946822000F00CF942
:1093F00038BD000058020020AC0800001CB5030C6A
:109400006A461370030A53709070080CD070080AF3
:109410001071517106226946942000F0F5F8024956
:10942000062048701CBD00005802002001B5FFF75F
:10943000B7FC01226946842000F0E6F801490020CB
:10944000487008BD5802002001B5012269468020FD
:1094500000F0DAF8684601780348002902D00221BA
:10946000417008BD0121FBE75802002001B501222F
:1094700069469F2000F0C8F808BD014610B51B20C2
:109480000822800100F0EAF8002010BD08B5074A64
:1094900004215170020C69460A70020A4A708870F1
:1094A0000322832000F0B0F808BD0000580200201D
:1094B00010B500221146D12000F0A6F810BD000022
:1094C000F8B504460D460020FFF7D0FC02271B4EDE
:1094D000FF43012809D00123002207210420FFF7C0
:1094E000B3FE162C19DD16241AE00F2C09D0012327
:1094F0001A4600210420FFF7A7FE0E2C08DB0E24DD
:1095000009E001231A4600210620FFF79DFEF6E739
:10951000BC4200DA3C46182103E0BC4200DA3C467B
:109520003821304600F094F86846047045700222F5
:1095300069468E2000F068F8F8BD0000E7080000DA
:1095400070B504460A488078002810D1D725ED0070
:109550002846FFF777FD4008E1054000C90F0143A9
:10956000284600F075F8E1B2681C00F071F870BD93
:109570005802002010B5044C04212046FCF784FF5B
:109580000128F9D010BD00000004005010B50A4CAD
:10959000002220212046FCF780FFC02000F0C2F806
:1095A000002000F0BFF8012220212046FCF775FFC3
:1095B000FFF7E0FF10BD000000040050F8B51546AD
:1095C0000E460446FFF728FC0E4F002220213846A5
:1095D000FCF763FF0E2000F0A5F8204600F0A2F88B
:1095E000002404E0305D00F09DF8641CA4B2AC429D
:1095F000F8D3012220213846FCF74FFFFFF7BAFFCE
:10960000F8BD000000040050F8B515460E460746A8
:10961000FFF702FC002220210C48FCF73EFF3846F1
:1096200000F080F8002404E0305D00F07BF8641C5A
:10963000A4B2AC42F8D3012220210448FCF72DFF4C
:10964000842F01D0FFF796FFF8BD00000004005002
:1096500013B5012201A900F001F81CBDF8B51546AB
:109660000E460446FFF7D8FB0F4F00222021384654
:10967000FCF713FF0D2000F055F8200A00F052F817
:10968000E0B200F04FF8002404E0305D00F04AF84A
:10969000641CA4B2AC42F8D3012220213846FCF766
:1096A000FCFEFFF767FFF8BD00040050F8B5044664
:1096B00000206A461080194D55222A70AA226A702D
:1096C0000322AA70661DEE702A716971144A49005E
:1096D0008918AC712246E81DFBF761FD002007E008
:1096E00029186A468978128889186A461180401CB0
:1096F000B042F5DB611DA81CFCF782F80146684604
:10970000018029190078C87168464078087221469E
:109710000931024800F03AFBF8BD00003C0E002081
:10972000800B002001B582B00021684601717D20C8
:10973000C0000090012301AA02A90348FDF754FCD0
:10974000684600790EBD0000AC140020034A116881
:10975000382389B2994301431160704700300140BA
:10976000F7B51A4D0446286B8AB00E468047184953
:1097700020464843E968884716480121C4820024EE
:1097800015480890079408200694029005940191CA
:109790000C980394009604940223EF6941B2224688
:1097A0000120B8470820069407940894099405946A
:1097B000029403940494009401900123AC6932460E
:1097C00002211846A0470DB0F0BD000020B00008EF
:1097D00040420F0060020020B80B000010B5FCF7FB
:1097E00069FE10BD10B59AB034216846FBF7F0FC55
:1097F000142114A8FBF7ECFC1C210DA8FBF7E8FCD6
:109800001D4801680324E402A143C21489180160C1
:10981000FCF7A4FF19480169A14301610E200090E3
:10982000FF20013002901020049002200990400493
:1098300001210B900001059100240C9003910A94E2
:109840006846FDF757F90F201490032015901694E1
:1098500017940121189414A8FDF73AF885200D906B
:10986000032080021190000213900F940DA8FCF7C2
:109870007DFF1AB010BD0000007000404010024093
:1098800010480168821511430160C1680E4A1140F9
:10989000C16001680D4A11400160816849084900B2
:1098A000816001680122920491430160C168FD2238
:1098B00012049143C1600021016106490448886097
:1098C00070470000001002400C40FF88F6FFF6FED3
:1098D0000050000800ED00E070B5026801239B070E
:1098E000114C124D984203D0A04201D0A84203D19E
:1098F0007026B2434E683243984203D0A04201D052
:10990000A84204D103231B029A43CB681A43802345
:109910009A430B691A4302608A68C26209688162CD
:109920000121416170BD00000008014000140140A8
:1099300030B5026A520852000262026A45688369C1
:109940007024A3439C080B68A40023430224A24371
:109950008C6845601443836149684163046230BD8B
:1099600030B5026A10239A430262036A456882692D
:1099700073242402A2430C6824021443202293433C
:109980008A68456012011A438461496881630262F2
:1099900030BD30B5026AFF2301339A430262026A86
:1099A0004568C3697024A3439C080B68A400234343
:1099B00001246402A2438C68456024021443C361FD
:1099C0004968C163046230BD30B5026A01231B03DC
:1099D0009A430262036A4568C26973242402A2435F
:1099E0000C68240214430122520393438A684560A1
:1099F00012031A43C46149680164026230BD000069
:109A0000F0B500211B4B0A4608469D7A2CE01A4E01
:109A1000345C631CDBB23354032C0ED2164C46006C
:109A2000B4463234A65B154F54003E536646C83FD9
:109A3000BE5B6437521C3E5392B25E1C0E4CF6B2B3
:109A400026541E2B0ED223464700BC463233DF5B22
:109A50004C001F5367466433DF5B1F53963B5E54D5
:109A6000491C89B2401C80B2A842D0D30148C272BE
:109A70008172F0BD6000002094100020F2110020DF
:109A800010B5818CC90707D001684A6801235B04BF
:109A90009A43836A1A434A60818C890707D5016813
:109AA0004A6801231B049A43C36A1A434A60818CA3
:109AB000490707D501684A6801239B049A43036B51
:109AC0001A434A60818C090707D501684A68012357
:109AD000DB039A43436B1A434A60818CC90607D55E
:109AE0000268916801231B039943836B19439160BA
:109AF000818C890607D501688A6801235B039A4334
:109B0000C36B1A438A60818C490612D503685A6870
:109B100001210905046C8A4322435A60026C8A427F
:109B200007D10268516803235B059943436C1943CD
:109B30005160818C090607D501684A680123DB045E
:109B4000806C9A4302434A6010BD0000F8B50026BD
:109B50000446C667FCF7A8FC054620680068124F5B
:109B6000000709D501212B46002249052046009710
:109B700000F0AAFA00280DD12068006840070BD534
:109B800001212B46002289052046009700F09CFA0F
:109B9000002801D00320F8BD20206067A067603452
:109BA00026740020F8BD0000FFFFFF01F8B5174C38
:109BB000C826E078002828D16079002825D1012026
:109BC0006071134D686B002700281DD0686BC82199
:109BD000081A14E00F48E168405C616988470E4844
:109BE0000E49008840000880E068401CE060E068A2
:109BF000C82800DBE760696BC820401A761EE16860
:109C0000814201D0002EE5DC6771F8BD30000020F4
:109C100000000240B80A0020B8000020C400002064
:109C200070B5224CE07800283FD1207900283CD143
:109C3000012020711E4EF16900250906002933DA42
:109C40002156625791420AD1F06940062CD5A0797D
:109C5000002829D0A5712089401C208124E0A17909
:109C6000002903D1A0710A2000F0F5FC0020205645
:109C7000CC2148430F494218206912181279B26268
:109C8000401C00222061A256CC235A4389588142AD
:109C90000ADC25612078401C207020780A2800D139
:109CA0002570A078401CA070257170BD3000002088
:109CB00000380140C002002010B5806A0022014631
:109CC00040314A834A82FDF7A0FB10BD70B5846A1B
:109CD000606FA56F2168896800260906002906DAE9
:109CE000212804D152200653204600F047F820686E
:109CF0008068400606D5222D04D15A2006532046FE
:109D000000F02CF8E06F10210843E0672046FDF7D3
:109D10007CFB70BD10B501460968806A0968890638
:109D200014D400225A210A5201680A68FF23013321
:109D30009A430A6001688A68520852008A60016882
:109D40008A6840239A438A6020218167FDF7ACFD31
:109D500010BD10B5806AFDF7E9FD10BD01680A6805
:109D6000FF2321339A430A6001688A68520852002F
:109D70008A602021816700210166704701680A68B6
:109D8000C0239A430A6020214167704770B5164C82
:109D9000E278002A0CD12279002A09D10122E2704E
:109DA0000025C82903DC0222A256002A01DCE57046
:109DB00070BD0123E356CC2253430C4AD1500123FA
:109DC000E356CC2673439B180A460146181DFBF741
:109DD000E6F96078401C607060780A2800D16570F0
:109DE000A078401EA070E2E730000020C0020020F2
:109DF00010B5014640318B8B846F0268222C04D051
:109E0000906908210843906110BD526A446D1A4060
:109E10002280426D921C42654A8B521E4A83498BB6
:109E20000029F1D101680A68FF2321339A430A60AF
:109E300001688A68520852008A60202181670021E7
:109E40000166FDF731FD10BD10B5014640318B8B29
:109E5000846F0268222C04D0906908210843906125
:109E600010BD526A1A40436D1A70426D521C426511
:109E70004A8B521E4A83498B0029F1D101680A6836
:109E8000FF2321339A430A6001688A68520852000E
:109E90008A602021816700210166FDF705FD10BD64
:109EA000F8B504462669A268E7693243666910205E
:109EB00000253E432368324378491E68784F3E4070
:109EC00016431E6023685A6803263603B243E668C9
:109ED00032435A602368A2698B4201D0266A32431A
:109EE0009E680B273F02BE4316439E606D4E23685B
:109EF0006D4AB3420CD1D2689207920F06D0012A64
:109F000038D0022A34D0032A20D11EE001201DE0DF
:109F1000664EB3420AD1D2680C26324026D0042ABB
:109F200028D0082A24D00C2A10D10EE08B420DD163
:109F3000D66803229202164018D001229202B61A65
:109F400018D0B61A14D0964200D10820564A0126DD
:109F5000403A574FF6038B4236D100280CD00228E6
:109F60000DD0042812D008281FD11CE00020EDE7F6
:109F70000220EBE70420E9E7FCF760FD08E0106849
:109F8000C00601D5384605E04A4803E0FCF776FDF7
:109F9000002873D0626851005118814205D811031E
:109FA000814202D303E03046F4E7012566E0010E6A
:109FB00006025008002330185941FBF7AFF803217F
:109FC0000902411A3C4A55E0E169B14232D103002D
:109FD00000F0EBF909070A0D06250606062B060018
:109FE000E3E7FCF72BFD1CE0FCF738FD19E01068F7
:109FF0006168C00602D54808304A01E0304A480886
:10A000008018FBF775F880B201462E4A103991424C
:10A01000CBD8511C01400007400F08432CE0FCF74F
:10A020002DFD616840004A08EAE76168012248089E
:10A030001204E5E7030000F0B8F909070A0D062647
:10A040000606062C0600B0E7FCF7F8FC1DE0FCF75E
:10A0500005FD1AE010686168C00602D54808C019FD
:10A0600002E014484A081018FBF742F880B2014693
:10A07000144A1039914298D82168C860002020669F
:10A0800060662846F8BDFCF7F9FC61684A0880184C
:10A09000EAE7616848088019E6E7000000480040E8
:10A0A000F369FFEF003801404010024000440040D7
:10A0B00000093D000024F400FFFC0F0000127A00AC
:10A0C0000048E801EFFF0000FFB581B017460E46DB
:10A0D00004460A9D09E0681C07D0FCF7E5F90499DD
:10A0E000401AA8420CD8002D0AD02068C169304619
:10A0F000884318D00020B842EDD0002005B0F0BD54
:10A1000020680168FF22A1329143016020688168C4
:10A1100049084900816020206067A0670020603402
:10A1200020740320EAE70120E5E7000010B50449A8
:10A130001020096808620248FDF768F910BD0000A8
:10A140002C140020F8B50025154C164E164F642827
:10A150000BD062281ED0602806D1258400F0C6FEF0
:10A16000642000F071FAFE60F8BD1048694608806E
:10A1700072B680210E48FBF7DBFB002804D00222D8
:10A1800069460B48FBF778FC62B60AA000F0ECF8D1
:10A19000A584E3E70248658440380580DEE70000D7
:10A1A000C00B00200400FA0500ED00E0AAAA0000A0
:10A1B000384A0008BDF8C8EBC9FDBCB6C4A3CABD87
:10A1C0000D0A000001490920887070473000002006
:10A1D00010B586B014216846FAF7FAFF0D4800243E
:10A1E00084840D48016B4908490001630A20FCF78B
:10A1F0009DFA0A48FDF7ECF8032040020090032086
:10A2000001900520694602940007FCF781F806B02A
:10A2100010BD0000A0000020001002402C140020FF
:10A2200010B50748018B49008184FDF725FFFEF733
:10A230003FF8C82203490448FDF778FA10BD000032
:10A24000A0000020B80A00202C140020F8B5414CD2
:10A2500000232178404A1D46082910D007294ED0F6
:10A26000062957D0052959D004295AD003295BD093
:10A2700000295DD001295FD0022961D062E0A17878
:10A2800000264A1F04E0344FBF5DFB189BB2761CCA
:10A290009642F8DB627927799B185B18E1785E18A3
:10A2A0006378F618F6198019C00723D0012A1DD04B
:10A2B000022A1FD128480078012802D10846FFF75A
:10A2C00041FF2648E178627840182349FAF767FF92
:10A2D00000F00CFE642000F0B7F9BFF34F8F214966
:10A2E0001F48C860BFF34F8F00BFFDE749081846FD
:10A2F000FFF7DCF92570E570A570A571F8BDA179AF
:10A300005054491CC8B2A071A178491F8842F5D1A8
:10A31000082001E0607007202070F8BDE070062082
:10A32000FAE760710520F7E7A070E5700420F3E715
:10A33000552807D10120EFE7AA2803D10220EBE737
:10A34000032803D02570E570A570F8BD03202070A8
:10A350002071F8BD57000020D80D0020800B002090
:10A360000400FA0500ED00E010B5024A024900F0D1
:10A37000F7F810BD89AD0008800200202021020CF2
:10A3800001D010211046020A01D0104608390209F6
:10A3900001D01046091F820801D01046891E4208CC
:10A3A00001D0881E7047081A704730B47446641E86
:10A3B0002578641CAB4200D21D46635D5B00E31848
:10A3C00030BC184702E008C8121F08C1002AFAD1A1
:10A3D00070477047002001E001C1121F002AFBD125
:10A3E0007047000038B504466D20694608706B461A
:10A3F000012207492E2000F021FC0649002C01D043
:10A40000054A00E0054A2E2000F0FEFB38BD0000A2
:10A4100006080000061800000706000007160000E6
:10A4200010B5002000F006F800220421362000F0CC
:10A43000EBFB10BD38B504466B46022200213620E6
:10A4400000F06AFBB3212300FFF7AFFF0E0F0815E2
:10A450003A3A3A3A1C273A3A2F34483A00216846A9
:10A46000017040784108490014E069460878800886
:10A470008000401C04E06946087880088000801C49
:10A4800008701DE0684602780A4048320270417840
:10A49000802001436846417012E0684602780A4015
:10A4A000027040784106490EF4E769464878022177
:10A4B000084303E069464878FD2108406946487032
:10A4C0006B4601220021362000F0B8FB012200ABD0
:10A4D00011463620013300F0B1FB38BD69460878DB
:10A4E000CF21084069462030CAE708B503216846F5
:10A4F0004170012101706B4602220021362000F0DC
:10A500009DFB0122D20306212D2000F07DFB0120BE
:10A5100000F09AF80120FFF78DFF08BD08B5020A88
:10A5200069464A7008706B46022204212D2000F013
:10A5300085FB0320694608706B46012206212D2009
:10A5400000F07CFB0020694608706B460122062162
:10A550002D2000F073FB0A212D2000F0C3FA08BD66
:10A56000F8B516460F460446002503E03946B047C5
:10A57000641C6D1C20780028F8D12846F8BD000026
:10A58000F8B54A002B4B520DD6182B4A0C460546FF
:10A59000142E2BDA002E12DA284BFAF725FE0022B1
:10A5A0001346FBF709F840D2002C03DA0124E40734
:10A5B00000253AE02046284337D0214C14E0214FB3
:10A5C0000B46F7403B402B4331D01C4BFAF70CFEB7
:10A5D00000221346FAF7F0FF27D2002C03DD0120FA
:10A5E0000005F0400419BC4300251EE0332E1EDC9C
:10A5F00033460027143BFF43DF40384217D00F4B50
:10A60000FAF79CFE00221346FAF7D6FF0DD2002C73
:10A610000ADD142E0CD03420811B01208840401903
:10A62000A84200D2641C0546BD4321462846F8BD19
:10A63000641CF9E701FCFFFF9C7500883CE4377E51
:10A640000000F03FFFFF0F007D2110B5C900484317
:10A6500000F001F810BD002140E000BF00BF00BFC6
:10A6600000BF00BF00BF00BF00BF00BF00BF00BFF2
:10A6700000BF00BF00BF00BF00BF00BF00BF00BFE2
:10A6800000BF00BF00BF00BF00BF00BF00BF00BFD2
:10A6900000BF00BF00BF00BF00BF00BF00BF00BFC2
:10A6A00000BF00BF00BF00BF00BF00BF00BF00BFB2
:10A6B00000BF00BF00BF00BF00BF00BF00BF00BFA2
:10A6C00000BF00BF00BF00BF00BF00BF00BF00BF92
:10A6D00000BF00BF00BF00BF00BF491C8142BCD308
:10A6E0007047000038B50446FFF79AFEFF22520378
:10A6F0000021282000F093FA0E4A0021282000F0C3
:10A700008EFA0220FFF796FE0D20FFF793FE042C31
:10A7100000D20424224600210A2000F080FA1020F2
:10A72000694608706B46012224212F2000F086FA2A
:10A7300038BD000000FF5F00FEB504460020019018
:10A7400000906079734940000E5A61782578491E5F
:10A750007148CFB20163042D77D0072D75D0002149
:10A760000291217801736C49E3790122920589698C
:10A77000002B6CD0914381616748217A4173217A23
:10A7800082698907890B0A4382610021042000F055
:10A7900046FA324661492E2000F036FA3846FFF775
:10A7A00021FE5F4E0522705D810040185D4943180F
:10A7B00007212B2000F042FA5B49029801220B1876
:10A7C0000B21282000F03AFA705D584980000A58A1
:10A7D0000C21282000F023FAE07955498000401828
:10A7E000A1794900425A0221272000F00DFA514870
:10A7F0007E00825B0421272000F006FAE079002821
:10A8000029D0A07804282CD028206946087220225C
:10A810000621272000F0F8F902AB0122262127208B
:10A8200000F00CFA444938014018E1788900425898
:10A830000821272000F0F3F9A17A601C627A09024E
:10A84000114313D016E000E001E0012188E7114335
:10A85000F608816190E764220621272000F0D4F9F0
:10A86000E0E71020694608720246D1E733490172D9
:10A87000090A4172417A007A0A0202432021272004
:10A8800000F0C2F92E4F0C2123203A6800F0C7F9DE
:10A89000F01982880421232000F0B6F9A07900285D
:10A8A0000BD0E0792749012243180021212000F034
:10A8B000C5F903200190012000902A07120F100112
:10A8C0000243607800218007000B024301980005D5
:10A8D00002430098400402432079C0064009024325
:10A8E0006079C00602431F2000F099F9A0786178D2
:10A8F0000123084302040848DB030261E1794903AC
:10A9000019430A4302610021082000F088F9002061
:10A91000FEBD0000CCAF0008840200200428000027
:10A9200074AF00080B000020290000207CAF000855
:10A930009CAF0008A8AF0008ACAF000841100000B1
:10A9400094AF00082B00002010B5044604213620E7
:10A9500000F0C8F80121C902002C01D0084300E032
:10A96000884302460421362000F059F910BD00004A
:10A970007CB505460420694608704B4C0020607584
:10A9800021462031206348710873A0836063A0636F
:10A9900000F0BCF8454E206002E000F0B7F82060FF
:10A9A000B042FAD10020FFF745FD41480078242845
:10A9B00001D9243806E00621FAF79AFB0622101A7C
:10A9C00040010843020601040A4301020A4302430C
:10A9D00000211E2000F023F96B46012200212420D3
:10A9E00000F02CF91E20FFF799FD86B2300AA07303
:10A9F0000420FFF793FD0006000E0DD002206946EB
:10AA0000087101AB012212212D2000F017F9A08B53
:10AA1000012109030843A08300F078F82060062094
:10AA2000FFF77CFD60600720FFF778FDA060F0066F
:10AA3000C00E207501D110202075C0B200F028F999
:10AA4000E80707D0FFF751FDA08B0121C902084399
:10AA5000A0830AE00521362000F02EF815490840B1
:10AA600002460521362000F0CFF80120FFF7E2FC76
:10AA70000021042000F036F8A0610021262000F01B
:10AA800031F815218903084302460021262000F0F1
:10AA9000C6F800222621362000F0B6F800F036F87D
:10AAA000206000207CBD0000840200203001CADE4E
:10AAB0000A000020FFFD000038B5094C89B280B2C1
:10AAC0006B46022200F028F8002806D1684640783C
:10AAD000010268460078081884B2204638BD00009C
:10AAE000FFFF000038B50024E44389B280B26B4612
:10AAF000042200F011F8002806D103216846435CC7
:10AB00002202D418491EFAD5204638BD10B50021BE
:10AB10000846FFF7E7FF10BD38B5002909D04024EB
:10AB200020436C462070C8B27F2906D8607002208E
:10AB30000AE069460870012006E0802420436C4644
:10AB40006070C809A0700320694600F0A5F938BDFF
:10AB500010B5024602492E2000F056F810BD000044
:10AB60000418000010B502460021182000F04CF82F
:10AB700010BD0000F8B50746002568460570B80707
:10AB8000204C2E4600280ADA8020694608706B4661
:10AB9000012200210D2000F051F801202073F80758
:10ABA0006946087821D006210843694608706B463B
:10ABB000012200210D2000F041F803210F20FFF7B2
:10ABC0007BFF8121C900084219D0402069460870E6
:10ABD0006B46012200210D2000F030F80020FFF725
:10ABE000B3FE00252673ED4309E0022108436946C0
:10ABF00008706B46012200210D2000F01FF8284646
:10AC0000F8BD0000A402002008B56B461A70120AB5
:10AC10005A7089B280B2022200F010F808BD38B52F
:10AC200000236C46E254120A5B1C042BFADB89B247
:10AC300080B22346042200F001F838BD38B58024E4
:10AC4000002909D0C02528436D462870C8B27F2945
:10AC500007D86870022009E0204369460870012087
:10AC600004E020436870C809A8700320694600F01A
:10AC70005DF938BD10B5054A8905126901430A43DB
:10AC800000210820FFF7CBFF002010BD8402002028
:10AC900038B504466B4601220E212B20FFF73CFFFE
:10ACA00068460078E10640094001C90E0143684644
:10ACB00001706B4601220E212B20FFF7BFFF38BD2C
:10ACC000F8B54A002B4B520DD6182B4A0C460546B8
:10ACD000142E2BDA002E12DA284BFAF785FA00220E
:10ACE0001346FAF769FC40D2002C02DB002425460B
:10ACF0003BE060004008284337D0214C14E0214F4E
:10AD00000B46F7403B402B4331D01C4BFAF76CFA13
:10AD100000221346FAF750FC27D2002C03DA012058
:10AD20000005F0400419BC4300251EE0332E1EDC54
:10AD300033460027143BFF43DF40384217D00F4B08
:10AD4000FAF7FCFA00221346FAF736FC0DD2002C73
:10AD50000ADA142E0CD03420811B012088404019BF
:10AD6000A84200D2641C0546BD4321462846F8BDD2
:10AD7000641CF9E701FCFFFF9C7500883CE4377E0A
:10AD80000000F0BFFFFF0F0013B501231A4669460C
:10AD90000248FCF7CCFD00981CBD00002C140020DC
:10ADA000FBF790FBFEF71EFDFDF766F9FDF778F95E
:10ADB000FDF77EFAFDF72CFAFDF728F9FDF74AFAC0
:10ADC0001348124901600021416081600162114A0B
:10ADD000416242618162FBF733FC012205201102CE
:10ADE0000007FBF75AFBFDF7BFFAFCF777FFFAF70E
:10ADF00037FD0948FFF776FC00210D20FFF73AFFE9
:10AE00000020FFF7B7FEFCF719FFFCE7007C0040CD
:10AE10007C130020FFFF000080E7010010B5FF2237
:10AE20002D321A491A48FAF79DFD18481949028827
:10AE30008A422AD0018004218180FF21F531C1801E
:10AE40000A21018100211E224181D24382810122F7
:10AE5000C281018401824182C182018381834323B3
:10AE6000C386022303877823438782870246C187EC
:10AE700040329180118451849184C183472109011A
:10AE800041841621818200F031F810BD800B002032
:10AE900000FC0008AA550000F0B58C4600251026DD
:10AEA000052109078E620E4C08E067467F5DE7606A
:10AEB000A768FF07FCD0E7681F706D1C8542F4DBB4
:10AEC0000020074606E0E760A568ED07FCD0E568CE
:10AED0001D54401C9042F6D38E610020F0BD00004E
:10AEE0000030014010B5FAF7FDFB10BD70B572B629
:10AEF000FF250B4E2D3529463046FAF719FD040083
:10AF000005D02A4607493046FAF7B6FD044662B630
:10AF1000962204490448FAF742F9204670BD000021
:10AF200000FC0008800B0020AC0C0020F0B50025D0
:10AF3000102605279C463F070B46BE620C4C06E0D8
:10AF4000595DE160A168C907FCD0E1686D1C8542CC
:10AF5000F6DB002007E06146095CE160A168C907F3
:10AF6000FCD0E168401C9042F5D3BE610020F0BDEA
:10AF7000003001400000010203040005405C0000B5
:10AF8000A05C0400C06C0800805C0400E03F1E0070
:10AF9000E07D1E0007A9022570889B880A00160024
:10AFA000010006000100020087008D002D001A310B
:10AFB00052001A339A001A351D011A376B003B31C3
:10AFC000BE003B335E013B3596023B37000099598A
:10AFD0009959EB518F421E45142E0080EB51F528F4
:10AFE0003333E13A703DE13AC235852BC235333314
:10AFF000C235C235AE47E13A5138A330513800006E
:10B000000000000000000102030406070809030411
:10B0100006080C1018203000000000010203040094
:10B02000ED840008C9840008718700083D87000886
:10B030001D8600084D860008D98700087189000820
:10B0400091840008E98A0008FD860008B58A000896
:10B05000D58A000899860008DF8A0008A18A0008BE
:10B06000918600086D8C000881860008758C0008A8
:10B070008986000845870008A1870008E784000842
:10B0800035850008CD86000869890008040506009A
:10B09000C01200001F000000A816000017000000EA
:10B0A000841C00000F000000E42500001E000000CA
:10B0B000B42D000016000000083900000E0000004A
:10B0C0002C4C00001D000000685B00001500000013
:10B0D000747200000D000000589800001C00000071
:10B0E00034B7000014000000E8E400000C00000089
:10B0F000783101001B000000686E010013000000A1
:10B1000034CA01000B000000286202001A0000008F
:10B1100040DB0200120000003C9303000A00000024
:10B12000C0C204001900000060B305001100000057
:10B13000382007000900000020A1070000000000DF
:10B1400060B100080000002084020000845700085D
:10B15000D8B10008840200207C190000D4A30008A4
:10B16000B1130704380D091E0805400826091040D0
:10B1700008560A131D043B08BE05061ED8BC401025
:10B180000814050214150909010262810215010360
:10B190002D0E0E0A1401460116BBC8423B0009C51C
:10B1A000020304050607080952200217FF4809FC9C
:10B1B000A9F1D24D624040085A30085A20085A106E
:10B1C000081159080B2CF03F285AE008092628E3FB
:08B1D000D03F12FF031A1A041C
:04000005080050C1DE
:00000001FF
